:020000040000FA
:020000000F28C7
:06000A0082074834753442
:100010006D3465346434613464343A3400348312AA
:100020000313850186018701831606309F00850131
:10003000860187018312850186018701D101003085
:10004000D300D400A02001309720063097200C3038
:10005000972080309720270805200038031933287F
:100060009B20A70A2B28D120B620C6205508612046
:10007000831203138930972003113108303A031D8E
:10008000442820309B204D2831089B200311310843
:10009000303A031D4D2820309B2032089B20330826
:1000A0009B2025309B2086013428C730A500000006
:1000B0000000A50B57280800A6005520A60B5D28B8
:1000C0000800B400B101B201B30164303402031C72
:1000D0006C28B400B10A65280A303402031C732866
:1000E000B400B20A6C283408B300B4013030B30451
:1000F000B204B10803197F283030B1040800303051
:10010000B1000800051500000000000005110800FE
:1001100085148316FF308600831205150000861BA8
:100120008F2805118316860183128510080005109B
:1001300086008820822805108600882005148228E1
:1001400038309720AA2038309720AA2038309720BE
:10015000AA2008000630A100CF30A2000000A20BA8
:10016000AE28A10BAC28B42800000800A730A100DD
:100170002930A2004830A3000000A30BBC28A20B2A
:10018000BA28A10BB828C42800000800192105309E
:1001900028213E2150215321732163218521912162
:1001A00008001921073028213E2153213E216321D7
:1001B00085211921063028213E2153145308282176
:1001C0003E2108001921073028213E2153213E21DC
:1001D000632185211921063028213E21531053081F
:1001E00028213E2108001921073028213E215321D2
:1001F0003E21632185211921063028213E215315F6
:10020000530828213E2108001921073028213E21CA
:1002100053213E21632185211921063028213E21C9
:100220005311530828213E21080019211E3028218E
:1002300008008316031306108610831206140000AC
:100240000000861406108610861406148610080016
:10025000D200D0010310831606108312D20D0318AA
:10026000352986100610861438298610061486143F
:100270000730500203190800D00A2E2983160614ED
:100280008312000000000000000086100000000043
:10029000000000000000861406184529861008009A
:1002A000061850290800D301531486108614061C22
:1002B0005E29D30D5314031C55290800D30D531088
:1002C000031C55290800D401541486108614061CFA
:1002D0006E29D40D5414031C65290800D40D541044
:1002E000031C652908008316061083128610061069
:1002F0008614000000000000000000000000000064
:100300000000831606148312080083160610831259
:1003100086100614861400008610831606148312B5
:1003200008000030E0005408E1006C30540203186B
:10033000AE298F30E3000030E200BC2103306402BC
:10034000031CA9290230E40203306402031CA9291A
:10035000B9290230E400E501B929B9296F30E30079
:100360000030E200BC210B30E4074D30E5070318F4
:10037000E40A6408D5000800DB210310E60CE70C52
:10038000031CC8296108E3070318E20A6008E207B2
:10039000E20CE30CE40CE50CE80BBE29E42969103F
:1003A0006108E3070318E20A031869146008E2070A
:1003B0006918031408001030E8006208E6006308BA
:0A03C000E700E201E3010800080075
:02400E00313D42
:00000001FF
